:1000000010C02AC029C028C027C026C025C024C0CF
:1000100023C022C021C020C01FC01EC01DC01CC0E4
:100020001BC011241FBECFE5D1E0DEBFCDBF10E065
:10003000A0E6B0E0E6E8F3E002C005900D92A23839
:10004000B107D9F720E0A2E8B0E001C01D92A03AC4
:10005000B207E1F72DD195C1D3CFDC01FA011082AF
:100060008C918623E9F789EF90E00197F1F700C0C2
:10007000000083EF91E00197F1F700C000008C9140
:10008000862319F080818160808383EF91E001975E
:10009000F1F700C000008C91862319F08081826006
:1000A000808383EF91E00197F1F700C000008C910D
:1000B000862319F080818460808383EF91E001972B
:1000C000F1F700C000008C91862319F080818860D0
:1000D000808383EF91E00197F1F700C000008C91DD
:1000E000862319F080818061808383EF91E00197FE
:1000F000F1F700C000008C91862319F080818062A6
:10010000808383EF91E00197F1F700C000008C91AC
:10011000862319F080818064808383EF91E00197CA
:10012000F1F700C000008C91862319F0808180686F
:10013000808383EF91E00197F1F700C0000089EF21
:1001400090E00197F1F700C000000895FC01908154
:10015000862F809598239083A3EFB1E01197F1F754
:1001600000C00000908140FF02C0962B01C0982380
:100170009083A3EFB1E01197F1F700C000009081E8
:1001800041FF02C0962B01C098239083A3EFB1E0FA
:100190001197F1F700C00000908142FF02C0962B3A
:1001A00001C098239083A3EFB1E01197F1F700C04D
:1001B0000000908143FF02C0962B01C098239083DA
:1001C000A3EFB1E01197F1F700C00000908144FF68
:1001D00002C0962B01C098239083A3EFB1E0119742
:1001E000F1F700C00000908145FF02C0962B01C0CE
:1001F00098239083A3EFB1E01197F1F700C00000BE
:10020000908146FF02C0962B01C098239083A3EFF4
:10021000B1E01197F1F700C0000047FF04C08081F2
:10022000862B808303C090819823908383EF91E095
:100230000197F1F700C000008081862B8083A3EF37
:10024000B1E01197F1F700C0000083EF91E0019752
:10025000F1F700C000000895FF920F931F93CF9312
:10026000DF938C01F62EEA0110929F0010929E00FF
:10027000E0919E00F0919F00EC0FFD1F40816F2DDB
:10028000C80164DF20919E0030919F002F5F3F4F97
:1002900030939F0020939E00FE01E20FF31F8081A8
:1002A0008111E6CFDF91CF911F910F91FF900895BB
:1002B00080E886BD16BCD99AD19A40E650E062E04B
:1002C0008BE390E0C9DF2FE784E89EE12150804076
:1002D0009040E1F700C0000040E650E062E08BE3B0
:1002E00090E0BADF40E650E062E08BE390E0B4DFFC
:1002F00040E650E062E08BE390E0AEDF40E650E0A5
:1003000062E08BE390E0A8DF40E650E062E08BE340
:1003100090E0A2DF10929D0010929C004BE950E00B
:1003200061E089E390E099DE40E650E062E08BE333
:1003300090E092DF20919C0030919D00C9010196D0
:1003400090939D0080939C00F901EE57FF4F4091E0
:100350009B004083489721F410929D0010929C00CE
:1003600042E850E062E08BE390E076DF42E262E058
:100370008BE390E0EBDE4AE062E08BE390E0E6DEC8
:06038000CDCFF894FFCF81
:1003860068656C6C6F2E667464692E34342E6563F2
:10039600686F2E633A20796F7520747970656420D2
:0203A600220033
:00000001FF
